:1000000009C021C020C020C01EC01DC01CC01BC014
:100010001AC019C011241FBECFE9CDBF10E0A0E661
:10002000B0E0E0E6F3E002C005900D92A236B10721
:10003000D9F720E0A2E6B0E001C01D92AC36B207CD
:10004000E1F796D08BC1DCCF1F920F920FB60F92C3
:1000500011242F933F934F935F936F937F938F93CD
:100060009F93AF93BF93EF93FF93809162008F5F55
:100070008093620090916000981708F045C086E078
:1000800080936000B39908C0809164008F5F809373
:1000900064008CE08093600080916400853010F0F3
:1000A00010926400B49908C0809166008F5F8093BD
:1000B00066008CE08093600080916600853010F0CF
:1000C00010926600B3991EC0B4991CC081E0809361
:1000D000640082E0809366006091640088E090E0B4
:1000E0002CD16091660080E190E027D1C098C29841
:1000F000C1982FE789EA93E0215080409040E1F7D2
:1001000000C0000010926200FF91EF91BF91AF918B
:100110009F918F917F916F915F914F913F912F911F
:100120000F900FBE0F901F90189580916300813043
:1001300059F038F0823059F0833071F4C098C29A87
:100140000AC0C09AC29807C0C09AC29802C0C0989C
:10015000C29AC19A01C0C198809163008F5F809359
:10016000630080916300843010F010926300089562
:10017000BC98BB98C49AC39AB89ABA9AB99A88E0BC
:1001800090E0D4D08093640080E190E0CFD0809361
:10019000660080916400853018F081E080936400EF
:1001A00080916600853018F082E08093660083B706
:1001B000826083BF83B7816083BF89B7826089BF54
:1001C00078948DE0E82E9AE0D92E28E0F22E38E2DD
:1001D000C32E44E1B42E54E0A52E09E010E0809136
:1001E0006400823091F038F4882361F0813091F41A
:1001F000B09267000FC0833059F0843059F4F09208
:10020000670008C0C092670005C0E092670002C0A6
:10021000D09267008091690090916700890F809368
:10022000690080916900853670F190916400809139
:10023000650098130CC09091660080916B00981334
:1002400006C0809168008F5F8093680002C01092A2
:100250006800809168008A3061F46091640088E0F1
:1002600090E06BD06091660080E190E066D01092E3
:10027000680080916400809365008091660080939F
:100280006B001092690080916600823089F030F432
:10029000882359F0813091F482E00EC0833059F008
:1002A000843061F4F0926A0009C010926A0006C0BE
:1002B000A0926A0003C086E080936A008091640087
:1002C000823091F038F4882361F0813091F4C0E7F6
:1002D000D7E10FC0833059F0843059F4C0E6D9E03B
:1002E00008C0C0EEDEE205C0C0EADFE002C0C8EB35
:1002F000DBE01BDF80E090916A00981728F0FE0198
:100300003197F1F78F5FF7CF10DF20E030916A006F
:10031000822F90E0A801431B5109841795070CF028
:100320005ECFCE010197F1F72F5FF0CFE199FECFBD
:100330008EBBE09A99278DB30895262FE199FECFC1
:100340008EBBE09A81500DB2021639F01CBA2DBB5B
:100350000FB6F894E29AE19A0FBE0895F894FFCF91
:02036000060095
:00000001FF
